:100000000AC018951895189518951895189518956B
:100010001895189518958FED8DBFC0ECE8EB4E2E16
:10002000DD275D2EEEE7F0E0A0E6B0E088278D93B7
:100030003197E9F7EDD266248FE087BB8FEF81BB64
:1000400080E082BB8FE788BB84E690E055D38CE0EC
:1000500027D3BF98A7E69C9197FF04C0B7990EC01D
:100060009F779C93B79B0AC088E29F93992744D3BC
:100070009F91B79B03C090689C9359D2AFD2EEE694
:10008000F7E0A4D2E2E0F0E0BAD2E9E0F0E0A6E6E0
:1000900091E066D3009166000E3C08F004C085B77D
:1000A000806385BF889580E080936400A1E637D3A4
:1000B00080E08093630080E0809365008FD2EEE75C
:1000C000F7E084D2C09AC39881E080936000BE9824
:1000D000A7E69C9196FF04C0B69B0EC09F7B9C93A5
:1000E000B6990AC088E29F93992706D39F91B69943
:1000F00003C090649C9313D182E080936000BD980C
:10010000A7E69C9195FF04C0B59B0EC09F7D9C9374
:10011000B5990AC088E29F939927EED29F91B5992D
:1001200003C090629C93FBD083E080936000BC98F6
:10013000A7E69C9194FF04C0B49B0EC09F7E9C9345
:10014000B4990AC088E29F939927D6D29F91B49917
:1001500003C090619C93E3D0C39AC29884E08093DB
:100160006000BE98A7E69C9196FF04C0B69B0EC0A7
:100170009F7B9C93B6990AC088E29F939927BCD233
:100180009F91B69903C090649C93C9D085E08093F9
:100190006000BD98A7E69C9195FF04C0B59B0EC07A
:1001A0009F7D9C93B5990AC088E29F939927A4D21A
:1001B0009F91B59903C090629C93B1D086E08093E3
:1001C0006000BC98A7E69C9194FF04C0B49B0EC04D
:1001D0009F7E9C93B4990AC088E29F9399278CD202
:1001E0009F91B49903C090619C9399D0C29AC19891
:1001F00087E080936000BE98A7E69C9196FF04C0BC
:10020000B69B0EC09F7B9C93B6990AC088E29F93D1
:10021000992772D29F91B69903C090649C937FD026
:1002200088E080936000BD98A7E69C9195FF04C08C
:10023000B59B0EC09F7D9C93B5990AC088E29F93A1
:1002400099275AD29F91B59903C090629C9367D029
:1002500089E080936000BC98A7E69C9194FF04C05D
:10026000B49B0EC09F7E9C93B4990AC088E29F9372
:10027000992742D29F91B49903C090619C934FD02B
:10028000C19AC0988BE080936000BE98A7E69C91CD
:1002900096FF04C0B69B0EC09F7B9C93B6990AC084
:1002A00088E29F93992728D29F91B69903C09064C2
:1002B0009C9335D08AE080936000BD98A7E69C911E
:1002C00095FF04C0B59B0EC09F7D9C93B5990AC055
:1002D00088E29F93992710D29F91B59903C09062AD
:1002E0009C931DD08CE080936000BC98A7E69C9105
:1002F00094FF04C0B49B0EC09F7E9C93B4990AC027
:1003000088E29F939927F8D19F91B49903C0906197
:100310009C9305D08AE090E0EFD1D4CE95CE939A0D
:1003200084E690E0E9D1939884E690E0E5D10091ED
:100330006400013009F001C048C00091640002303F
:1003400009F001C067C0009160000B3009F02AC0BD
:10035000A6E30C9104FB81E00EF480E08F93A6E30A
:100360000C9105FB81E00EF480E09F91892B8F9327
:10037000A6E30C9106FB81E00EF480E09F91892BAF
:10038000882309F401C0E4CF29D1ECE8F7E01ED1BD
:10039000A4E68C918F5F8C9380E0809363008FE75D
:1003A00088BB90CE009160000C3009F00DC0EAE0EF
:1003B000F0E0A4E1D4D1A1E60D911C91041715073A
:1003C00009F001C091C069C03AC0009160000C30D2
:1003D00009F01FC0EAE0F0E0A4E1C1D1A1E60D916F
:1003E0001C910417150709F401C057C0A1E697D165
:1003F00080E08093630080E080936500A4E68C91A8
:100400008F5F8C93EBD0ECE9F7E0E0D08FE788BB0F
:1004100059CE15C0009160000C3009F010C0EAE020
:10042000F0E0A1E67BE78AD1D9D0ECEAF7E0CED0C4
:100430004AD0E2E0F0E0E3D08FE788BB26CEA3E627
:100440008C918F5F8C930091630045E0040FA5E6CB
:100450000C938FEBA5E61C91D0D0ECEBF7E0B6D077
:1004600000916300063010F009F001C001C015C012
:10047000A1E60D911C914AE050E095D0A1E60D93C4
:100480001C93A1E60D911C91A0E64D915527040FF8
:10049000151FA1E60D931C930895A0D0EEEBF7E095
:1004A00095D084E690E028D18FE788BB939AE3E06B
:1004B000F0E0A5D0939890D0EEE6F7E087D0E4E1A5
:1004C000F0E09DD0E2CD84E690E016D1939A88ECDE
:1004D00090E012D1939888EC90E00ED1939A88EC3A
:1004E00090E00AD19398089580916600815080939E
:1004F0006600E9E0F0E0A6E691E07BE720D16ED06F
:10050000ECEAF7E063D0DFDF67D0ECECF7E05ED039
:100510008CE291E0F1D08FE788BB949AE1E0F0E0C3
:100520006ED094985BD0E1E0F0E069D0AECDE1E030
:10053000F0E065D0B79901C014C0EAE0F0E002ED48
:1005400014E0A0E1BB277BE7F9D0BDDF47D0EAED9F
:10055000F7E03CD041D0EAEEF7E038D0E5E0F0E05B
:100560004ED093CD04D01FD000FC0CD008950024B1
:10057000E89457FF02C009D0689400F80BD010F837
:100580000124089502D009D00895509540954F5FF9
:100590005F4F0895E89417FF0895009510950F5F39
:1005A0001F4F68940895752F642F55274427FF9394
:1005B000F1E1889405C010F4460F571F56954795F2
:1005C00017950795FA95B9F7FF910895A4D0802D56
:1005D00011F060D0FBCF089580EC62C081E060D064
:1005E00014D080E85DC08FE7213039F08FEB2230E6
:1005F00021F08FE8233009F08FEC810F51C088EE95
:1006000093E07AD03197D9F7089583E0992774C0A1
:100610008AEF90E071D0BB9ABA9AB99AB89A8E9A3A
:100620008D9A959885E090E067D09698C398C29887
:10063000C19AC09A969AEF93FF93E0E6F0E050D00B
:10064000FF91EF91969855D0969AEF93FF93E0E63D
:10065000F0E046D0FF91EF9196984BD0969AEF93A9
:10066000FF93E0E6F0E03CD0FF91EF91969841D007
:10067000C098969AEF93FF93E0E6F0E031D0FF91B7
:10068000EF91969836D088E20BD08EE009D086E0C4
:1006900007D00895959A829505D004D02AD0089560
:1006A0009598F9CF859510F4C09A01C0C0988595AA
:1006B00010F4C19A01C0C198859510F4C29A01C086
:1006C000C298859510F4C39A01C0C398969AEF9387
:1006D000FF93E0E6F0E004D0FF91EF919698089543
:1006E0003197F1F70895689462F80895E89462F8F4
:1006F000089581E090E000C0EF93FF93EE27E82B90
:10070000E92B31F0E8EEF3E03197F1F70197D1F7FB
:10071000FF91EF910895C89531960020089582E0E9
:1007200001C084E099279D938A95E9F70895E1999E
:10073000FECFEEBB3196089591E001C092E07B3789
:1007400051F47FB7F894F3DF8D918DBBE29AE19A73
:100750009A95C9F77FBF7727089591E001C092E08D
:10076000E6DFE09A8DB38D939A95D1F708955757A8
:10077000572E4156522E344D472E434F4D002020C8
:1007800020456E74657220636F64650020456E7449
:100790006572206F6C6420636F64650020456E7421
:1007A0006572206E657720636F64650020436F6417
:1007B0006520616363657074656400002A00202011
:1007C00020436F64652077726F6E670020202020C1
:1007D000556E6C6F636B656400002020496E697410
:1007E00069616C20636F646500002020202020690F
:0A07F0007320202031323334000062
:00000001FF
